:100000008C286400112003180128422008308F003A
:10001000432011208E0C0C288F0B082843200E083B
:100020000800240884002208841780048413000533
:1000300021192206FF3E080092002408840009309E
:10004000930003102820920C930B222803142828D5
:100050008413A11D372800082204211D22068000D8
:10006000841700082204031C22068000432800088D
:100070002204031C2206211922068000841722096B
:10008000800543282117210D06398C0051208D0051
:100090008C0A5120211F6B2821138C0002308220F2
:1000A0006B2800308A000C08820701347534033451
:1000B000153400343C340C34D9348F018E00FF30B9
:1000C0008E07031C8F07031C872803308D00DF3049
:1000D0006B205F288D01E83E8C008D09FC30031CED
:1000E00074288C07031871288C0764008D0F712801
:1000F0000C187A288C1C7E2800007E28080003102B
:100100008D0C8C0CFF3E03187F280C088728831366
:1001100003138312640008008316033085008601F0
:1001200083120511B220B220051505116400051CCB
:10013000962805120530A4000830A2000630A10060
:1001400021301C200530A4000230A2000630A1009E
:100150000120A600FF30A606260886000515051119
:1001600005169628051201308F00F4305E20051622
:1001700001308F00F4305E200800FF3FFF3FFF3F5B
:08400000FF3FFF3FFF3FFF3FC0
:02400E00F53F7C
:00000001FF
